:100000000C947D020C94C1020C94C1020C94C102A8
:100010000C94C1020C94C1020C94C1020C94C10254
:100020000C94C1020C94C1020C945F140C94311511
:100030000C9493220C94C1020C94C1020C94C10242
:100040000C94C1020C9423030C94C1020C94C102C1
:100050000C94C1020C94FB220C94C1020C94C102BA
:100060000C94C1020C94C1020C94C1020C94C10204
:100070000C94C1020C94C1020C94C1020C94C102F4
:100080000C94D40A0C94C1020C94C1020C94C102C9
:100090000C94C1020C94C1020C94C1020C94C102D4
:1000A0000C94C1020C94C1020C94C1029E15C0159F
:1000B000AE16C015AE1605162816AE167D1690168D
:1000C0007A197A19A919A919E819081A5E1B5E1B71
:1000D000131A5E1BC31AC31A2A1B331B5E1B581B41
:1000E000D01AD01AD01AD01AD01AD01AD01AD01AC0
:1000F000D01AD01AD01AD01AD01AD01AD01AD01AB0
:10010000E01AEE1AF51AFC1A061B07634236B79B73
:10011000D8A71A39685618AEBAAB558C1D3CB7CC67
:100120005763BD6DEDFD753EF6177231BF000000DF
:10013000803F08000000BE922449123EABAAAA2AC2
:10014000BECDCCCC4C3E00000080BEABAAAAAA3EDD
:1001500000000000BF000000803F00000000000819
:100160004178D3BB4387D1133D190E3CC3BD4282B6
:10017000AD2B3E68EC8276BED98FE1A93E4C80EF74
:10018000FFBE01C4FF7F3F00000000000000000030
:1001900000000000000000010204060A0F17202CD6
:1001A0003A4A5D71879DB3C7DAE9F5FCFFFCF5E9D2
:1001B000DAC7B39D87715D4A3A2C20170F0A0604EF
:1001C0000201000000000000000000000000018C9F
:1001D000028CF1A242070C0310022A041B074507F8
:1001E0002D010B0116013E033B013B0327010B03CD
:1001F0001603400741071B032D022A032E021D018F
:100200001C011501290014001A0008001500170030
:100210001C0018000C001200130002202A00040029
:100220001600070009000A000B000D000E000F0069
:10023000330034002B001D001B00060019000500D0
:100240001100100036003700380028004C00E00094
:100250000000E100E2002C000000500051005200BC
:100260004F0000004C0027001E001F00200021004E
:1002700022002300240025002600012012000A008D
:100280001600180017001B207000430044004000B7
:10029000410042002B000420052006203A000720E0
:1002A0006D006E0072006F0071000920360037008B
:1002B00015000B2003202C000C203B0008203C00E4
:1002C00069000000290019201A2000000000000029
:1002D000000000000000000000000000000000001E
:1002E00000000000000000000000000000001320DB
:1002F00014201520060000001620052000001720FD
:1003000000000000000000000D2000000E200F2063
:100310001020112003202C00122000000000730088
:100320000000000028035400680065002000500011
:100330006C0061006E0063006B0020004B006500E4
:10034000790062006F0061007200640000002C03FD
:100350004F007200740068006F006C0069006E004E
:1003600065006100720020004B00650079006200AA
:100370006F00610072006400730000000403090450
:1003800009026D00040100A0FA0904000001030144
:100390000100092111010001223F00070581030826
:1003A000000A0904010001030102000921110100F2
:1003B00001224D000705820308000A09040200011A
:1003C0000300000009211101000122360007058306
:1003D0000308000A090403000103000000092111B9
:1003E00001000122390007058403100001120110E9
:1003F0000100000008EDFE6060010001020001053F
:10040000010906A101050719E029E7150025019555
:1004100008750181020508190129059505750191E5
:10042000029501750391010507190029771500252B
:1004300001957875018102C005010980A10185023D
:1004400016010026B7001A01002AB70075109501A1
:100450008100C0050C0901A1018503160100269C3D
:10046000021A01002A9C02751095018100C0050145
:100470000902A1010901A1000509190129051500B9
:10048000250195057501810295017503810105011D
:10049000093009311581257F9502750881060938D3
:1004A0001581257F950175088106050C0A3802150E
:1004B00081257F950175088106C0C005010906A147
:1004C00001050719E029E715002501950875018147
:1004D0000295017508810105081901290595057521
:1004E0000191029501750391010507190029FF1576
:1004F0000025FF950675088100C011241FBECFEFAF
:10050000DAE0DEBFCDBF04B603FE24C080911E0337
:1005100090911F03A0912003B09121038730904B4D
:10052000A740B04BB9F410921E0310921F03109213
:1005300020031092210314BE84B7877F84BF88E113
:100540000FB6F89480936000109260000FBEE0E058
:10055000F8E3099511E0A0E0B1E0E0E8F9E502C0B8
:1005600005900D92A03CB107D9F713E0A0ECB1E0E3
:1005700001C01D92AE31B107E1F70E94A5110C94A4
:10058000BE2C0C9400000895089581E0089508950C
:100590000C94C4020C94C5020C94C7020E948828D3
:1005A00023E030E0281B3109220F2093C401089575
:1005B000282F2F9880918000211108C0877F809379
:1005C000800010928D0010928C001BC08860809378
:1005D0008000233019F48FEF9FEF0FC083E090E08D
:1005E000821B9109880F991F2FEF3FEFA90102C0CD
:1005F000569547958A95E2F7CA0190938D008093AE
:100600008C000C94CE020E94CE0284E08093C30141
:100610001092C0010895279A2F988FEF9FEF909323
:100620008700809386008AE08093800089E1809330
:1006300081000E94F1270C9403030E940B036E9A21
:10064000769A0C94C3021F920F920FB60F92112448
:100650002F933F938F939F93EF93FF93E091C1016B
:10066000F091C201CF0101969093C2018093C10124
:100670000090C30102C0F695E7950A94E2F7EF7384
:100680008091C001823019F4E03251F404C081300D
:1006900039F4EF3329F480916F008D7F80936F00E0
:1006A000F0E0E457FE4FE49121E031E0E29FC00129
:1006B000E39F900D11240090C40102C09695879588
:1006C0000A94E2F790938D0080938C00FF91EF9154
:1006D0009F918F913F912F910F900FBE0F901F9080
:1006E000189581E008950C94710308950C941D03EE
:1006F00080911502882309F448C08091D10190911E
:10070000D201009779F40E94C5229093D201809380
:10071000D1018091D30190E0009771F48091D401D0
:1007200090E00AC00E94D122209100013091010185
:100730002817390740F329C00197880F991F880FA0
:10074000991FFC01EB52FE4F608171818281938180
:100750000E943A0AE091D30184E0E89FF00111245D
:10076000EB52FE4F60817181828193814FE050E0B6
:100770000E94F20D8091D30190E001966091D40126
:1007800070E00E946E2C8093D3010C94C8021092EA
:1007900017020C94070A0895089581E080931702C8
:1007A0000C94CC03089508958F929F92AF92BF92BC
:1007B000EF92FF920F931F93CF93DF93CDB7DEB7E6
:1007C000A3970FB6F894DEBF0FBECDBF7C01FC012E
:1007D00000811181C8010E94C220B8010E94D90580
:1007E0008C01B7010E947303882309F4CCC1003245
:1007F000F0E51F0741F4F7018281882309F458C00E
:100800000E94560EC0C10132F0E51F0741F4F70106
:100810008281882309F44CC00E945F0EB4C1023269
:10082000F0E51F0751F4F7018281882309F440C0E5
:100830000E94520E8111F0CFE3CF0332F0E51F0783
:1008400039F4F7018281882399F10E94CD039BC17D
:100850000432F0E51F0739F4F7018281882341F162
:100860000E94C70390C10532F0E51F0749F4F70164
:1008700082818823E9F0809117028111F1CFE5CFC1
:100880000632F0E51F0739F4F7018281882381F0F1
:100890000E94660E0AC00732F0E51F0749F4F7010F
:1008A0008281882329F00E94710E0E94D3036BC1BC
:1008B00080911702811105C0F70182818111CFC09B
:1008C00018C1003E110579F4F7018281882309F4EB
:1008D0004DC00E94070A81E0809316021092150213
:1008E0001092D40150C1023E110559F4F7018281E2
:1008F0008823E1F10E94070A109216021092150255
:1009000042C1033E110591F4F7018281882371F100
:100910000E94070A1092160281E08093150210923D
:10092000D3011092D2011092D1012DC102351105CF
:1009300059F4F7018281882309F425C180910001CF
:10094000909101010A970DC00135110579F4F70165
:100950008281882309F417C18091000190910101DF
:100960000A9690930101809300010DC1409104010A
:1009700083E2EFE1F1E0DE01119601900D928A959C
:10098000E1F7F701808121E030E02C0F3D1F280FB7
:10099000311DC9012091020130910301FC01E20FD8
:1009A000F31F6081772767FD7095640F711D88279D
:1009B00077FD8095982F0E94902920E030E040E458
:1009C00051E40E94F5284B015C01F701218184E08C
:1009D00090E0821B9109BC01882777FD8095982FB4
:1009E0000E9490299B01AC01C501B4010E948D2891
:1009F0009B01AC0160E070E080E090E40E94032B7A
:100A000020E030E04CED50E40E94A02A4B015C0154
:100A1000F70182818823D1F04FE050E0C501B40195
:100A20000E94F20D809116028823A1F08091D401DA
:100A300024E0829FF0011124EB52FE4F80829182CC
:100A4000A282B3828F5F8093D40104C0C501B40138
:100A50000E943A0A0F3F110508F02ECF94C08091F2
:100A6000D00181111FC0043130E5130709F051C0D6
:100A70000E94750381E08093D0010E94C52290936B
:100A8000CF018093CE011092C7011092C90110923C
:100A9000C8011092CB011092CA011092CD011092A0
:100AA000CC0171C08091CE019091CF010E94D122E2
:100AB000883C910570F48091C701E82FF0E0EE0FBB
:100AC000FF1FE853FE4F118300838F5F8093C701A0
:100AD0005AC0043880E5180721F00538104501F1A7
:100AE0003AC0F7018281882341F01092C50182E06B
:100AF0001EC0043830E5130759F58091C5018111F6
:100B000006C086E20E941E1886E20E94E61882E075
:100B10001CC00438F0E51F0741F305381045D9F42F
:100B2000F7018281882331F01092C60180E20E9491
:100B3000351929C08091C601811106C087E20E9443
:100B40001E1887E20E94E61880E20E943C191BC032
:100B50000538104529F381E08093C5018093C601D3
:100B6000C701A3960FB6F894DEBF0FBECDBFDF91CD
:100B7000CF911F910F91FF90EF90BF90AF909F90FA
:100B80008F900C94CA0280E0A3960FB6F894DEBF53
:100B90000FBECDBFDF91CF911F910F91FF90EF90CE
:100BA000BF90AF909F908F90089580E090E008955F
:100BB00008959CE0799FF001112490E3899FE00D56
:100BC000F11D1124E60FF11DEE0FFF1FEC5FFD4F2D
:100BD000859194910895880F991FFC01E45BFF4F64
:100BE000859194910895880F991FFC01E453FE4F5D
:100BF0008591949108950F931F93CF93DF93EC0108
:100C0000811521E39207A0F5C11580E3D80708F00C
:100C1000D7C0C83ED105D8F4C03ED10508F007C200
:100C2000C83AD10578F4C53AD10508F06AC0C13098
:100C3000D10509F463C008F4F7C1C430D10508F048
:100C4000F6C1F2C1CB3BD10508F466C0EDC1C115B8
:100C500090E2D90708F0AFC0C11521E0D20708F033
:100C6000E6C1C03FD10508F4DFC18E0110651FC287
:100C7000C03880E5D80700F5C03790E5D90708F0FF
:100C8000A3C0C11520E5D20709F4ACC050F4CE01D1
:100C9000905480319F4008F0C7C1DF708E01106A08
:100CA00006C2C13080E5D80709F4AEC0C43190E572
:100CB000D90708F4AFC0B8C1C33820E5D20709F49A
:100CC0008EC050F4C13890E5D90709F482C008F00D
:100CD00083C000E011EDEBC1C03181E5D80708F415
:100CE000A3C1C11597E5D90708F436C1CE019057C5
:100CF0008115904108F098C1DF7093C101E010E0C8
:100D0000D6C1C53AD10509F494C1C63AD10509F056
:100D100093C102E810E4CBC1C83AD10509F48FC1F0
:100D2000C93AD10509F48EC1CA3AD10509F48DC179
:100D3000CB3AD10509F48CC1CC3AD10509F48BC169
:100D4000CD3AD10509F48AC1C03BD10509F489C166
:100D5000CE3AD10509F488C1CF3AD10509F487C14B
:100D6000C13BD10509F486C1C23BD10509F485C157
:100D7000C33BD10509F484C1C43BD10509F483C147
:100D8000C53BD10509F482C1C63BD10509F481C137
:100D9000C73BD10509F480C1C83BD10509F47FC127
:100DA000C93BD10509F47EC1CA3BD10509F47DC117
:100DB00000E014E47CC1CE019F700E94F30578C16D
:100DC000DD278E01106C73C1CF70DD278E01146D8D
:100DD0006EC100E010ED6BC100E012ED68C100E0F3
:100DE00013ED65C10E94C91B0E94070A0E94CB0334
:100DF0008FEF94E32CE0815090402040E1F700C059
:100E000000000E94202353C18091F20281608093F0
:100E1000F2024DC10E948123811102C00E945D2314
:100E20000E94942390E090931D0380931C03C23092
:100E300080E5D80721F480911C03816086C0C4300E
:100E400090E5D90721F480911C0382607EC0C630F2
:100E500020E5D20721F480911C03846076C0C8305D
:100E600080E5D80719F480911C0327C0CA3090E5AB
:100E7000D90721F480911C03806167C0CC3020E544
:100E8000D20721F480911C0380625FC0CE3080E5E0
:100E9000D80721F480911C03806457C0C03190E5CD
:100EA000D90721F480911C0380684FC0C23120E52E
:100EB000D20729F480911C038460886046C0C33047
:100EC00080E5D80721F480911C038E7F3EC0C53099
:100ED00090E5D90721F480911C038D7F36C0C7307F
:100EE00020E5D20721F480911C038B7F2EC0C930EE
:100EF00080E5D80719F480911C0326C0CB3090E51B
:100F0000D90721F480911C038F7E1FC0CD3020E5CE
:100F1000D20721F480911C038F7D17C0CF3080E56C
:100F2000D80721F480911C038F7B0FC0C13190E55D
:100F3000D90721F480911C038F7707C0C331D045B6
:100F400031F480911C038B7F877F80931C038091F9
:100F50001C030E949823ABC08D2F99278F7099276F
:100F600081309105D9F49E012370332702C0880F88
:100F7000991F2A95E2F79C688E0144E0000F111F2B
:100F80004A95E1F700271370802B912B53E0CC0F8B
:100F9000DD1F5A95E1F7C076DD272FC0823091051D
:100FA00031F4DC2FCC278E01016F106A80C08330B2
:100FB000910569F4CE018370992701E010E002C029
:100FC000000F111F8A95E2F7C8019C680FC084309A
:100FD0009105B9F4CE018370992701E010E002C0B9
:100FE000000F111F8A95E2F7C8019A6823E0CC0F21
:100FF000DD1F2A95E1F7C07ED7708C010C2B1D2BCD
:1010000056C08530910531F4DC2FCC278E01046F5A
:10101000106A4DC0069709F04AC0CF71DD27DC2F5A
:10102000CC278E01106243C000E010E040C08E016A
:101030003EC001E810E43BC003E810E438C002EE13
:1010400014E435C009EE14E432C00AEE14E42FC0F3
:1010500005EB14E42CC006EB14E429C007EB14E400
:1010600026C00CEC14E423C00DEC14E420C003E80B
:1010700015E41DC00AE815E41AC002E915E417C01A
:1010800004E915E414C001E216E411C003E216E419
:101090000EC004E216E40BC005E216E408C006E246
:1010A00016E405C007E216E402C00AE216E4C8012D
:1010B000DF91CF911F910F9108959CE0799FF001EE
:1010C000112490E3899FE00DF11D1124E60FF11D1D
:1010D000EE0FFF1FEC5FFD4F85919491803E9105CF
:1010E000E0F4803C910558F58133910509F46FC017
:1010F00048F48932910509F463C08A32910509F4F4
:101100006DC072C089339105E9F082389105D1F044
:101110008533910509F44DC067C0833E910581F187
:1011200038F4803E9105B9F0823E9105D9F05CC05B
:10113000863E910561F1873E9105A1F155C00E945F
:10114000EB05089520911C0320FD02C021FF4CC037
:1011500080EE90E049C080911C0380FFF9CF89E3C5
:1011600090E042C080911C0382FF0EC080911C035E
:1011700084FF03C080E090E037C083EE90E034C08D
:1011800080911C0382FFF2CF82EE90E02DC080910F
:101190001C0383FF0BC080911C0384FDEBCF87EE03
:1011A00090E022C080911C0383FFF5CF86EE90E093
:1011B0001BC080911C0385FF07C089E290E014C02A
:1011C00080911C0385FFF9CF85E390E00DC08091ED
:1011D0001C0386FF07C08AE290E006C080911C03D2
:1011E00086FFF9CF81E390E00E94FB0508950C94FF
:1011F000CC02E82FF0E0E25BFE4F8081E82FEF7039
:10120000F0E082958F7021E030E0A90102C0440F28
:10121000551F8A95E2F740A308950F931F93CF932C
:10122000DF9385B7806885BF85B7806885BFC3E0D9
:10123000D0E001E010E0FE01E25BFE4F8081E82F8C
:10124000EF70F0E021A182958F70A80102C0440FD9
:10125000551F8A95E2F7CA01822B81A38C2F0E9429
:10126000F908219740F78BE090E061E070E0FC0125
:10127000EE5BFE4F2081E22FEF70F0E042A122955D
:101280002F70DB0102C0AA0FBB1F2A95E2F79D0158
:10129000242B22A3019758F7DF91CF911F910F9133
:1012A0000C947603EF92FF920F931F93CF93DF93EB
:1012B00000E212E0C3E0EE24E394F12CD5E08C2FA1
:1012C0000E94F9088BE090E040E050E0FC01EE5B0A
:1012D000FE4F6081E62FEF70F0E020A130E06295D4
:1012E0006F7002C0359527956A95E2F720FD09C019
:1012F0009701082E02C0220F331F0A94E2F7422BF7
:10130000532B019718F7F801929182918F0184175E
:10131000950721F051834083D09305018C2F0E94C3
:10132000F908C15060F68091050187FD2CC08150FD
:10133000809305018F3F39F08FE99FE00197F1F726
:1013400000C0000020C080911E0290911F02909367
:1013500027028093260280911C0290911D02909397
:1013600025028093240280911A0290911B0290938F
:101370002302809322028091180290911902909387
:101380002102809320020E94780381E0DF91CF91B7
:101390001F910F91FF90EF900895E82FF0E0EE0F6E
:1013A000FF1FE05EFD4F80819181089508950F93A6
:1013B0001F93CF9308E212E0C0E0F801929182916E
:1013C0008F010E943D22C80FF2E000321F07A9F7EB
:1013D0008C2FCF911F910F9108950E94812381112D
:1013E00002C00E945D230E94A623809307033E9AB9
:1013F000809171008D7F8093710082E080939000D6
:101400008AE18093910081E080932A02089580917F
:101410002A02811102C00E94ED0910927A021092F4
:101420007902809171008D7F80937100809190008E
:101430008F738093900010923C0210923B021092A6
:10144000730210927402109275021092760210923A
:10145000720210927102E1E5F2E0A1E4B2E01192B1
:101460001192119211921D921D9282E0E137F807BC
:10147000B1F70895CF92DF92EF92FF920F931F93EF
:10148000CF93DF9320913B02222309F484C06B01A8
:101490007C0180912A02811102C00E94ED0901E7BE
:1014A00012E0C7E0D0E0A7019601F8019291829185
:1014B000729162918F010E94F128811131C0FE0169
:1014C000EE0FFF1FEE0FFF1FEF5AFD4F108211822C
:1014D00012821382DE01AA0FBB1FAF5BBD4F1196B4
:1014E0001C921E92C730D105E9F0219644815581A6
:1014F000668177814083518362837383148215826E
:101500001682178212968D919C91139711969C9337
:101510008E9313961C921E92129734961296E2CFD7
:10152000219708F68091790290917A02019797FDB0
:1015300005C090937A028093790204C010927A02D7
:10154000109279028091790290917A02209177022B
:10155000309178022817390724F0109278021092FF
:101560007702892BC1F4809171008D7F8093710087
:10157000809190008F73809390001092730210926C
:1015800074021092750210927602109272021092FA
:10159000710210923B02DF91CF911F910F91FF904A
:1015A000EF90DF90CF9008951F920F920FB60F9299
:1015B00011244F925F926F927F928F929F92AF927F
:1015C000BF92CF92DF92EF92FF922F933F934F9370
:1015D0005F936F937F938F939F93AF93BF93CF93BB
:1015E000DF93EF93FF9380913B02882309F49BC123
:1015F000C0917902D0917A021C161D060CF093C19D
:1016000040902B0250902C0260902D0270902E0280
:1016100020E030E0A901C301B2010E949C2A181603
:101620000CF065C0C130D10509F452C08091770239
:1016300090917802BE010E946E2C7C0190937802FA
:101640008093770280903D0290903E02A0903F02EE
:10165000B090400220E030E040E85FE3C501B40113
:101660000E948D2860933D0270933E0280933F025A
:1016700090934002F701EE0FFF1FEE0FFF1FEF5A8E
:10168000FD4FA301920160817181828193810E944B
:10169000F52820E030E040E05EE30E94A02A9B01B4
:1016A000AC01C501B4010E949C2A18168CF4C70134
:1016B0000196BE010E946E2C90937802809377026F
:1016C00010923D0210923E0210923F021092400290
:1016D000E0917702F0917802EE0FFF1FEE0FFF1FEF
:1016E000EF5AFD4F6081718182819381D0C0C0909B
:1016F0007302D0907402E0907502F090760220E0C0
:1017000030E0A901C701B6010E94F1282197882382
:1017100009F4A2C0FE01EE0FFF1FEE0FFF1FEF5AEC
:10172000FD4F80809180A280B380A5019401C70104
:10173000B6010E94F12887FF31C0A501940160E045
:1017400070E08CED93EC0E94F52820E030E040E45E
:1017500051E40E94F52820E030E040E05FE30E9481
:10176000A02A9B01AC0160E070E080E090E40E9460
:10177000032B9B01AC01C501B4010E94A02A9B016F
:10178000AC01C701B6010E94F12887FF07C0A7017D
:10179000960160E070E08CED93E439C0A5019401FE
:1017A000C701B6010E949C2A18160CF055C0A5016D
:1017B000940160E070E08CED93E40E94F52820E055
:1017C00030E040E451E40E94F52820E030E040E0C1
:1017D0005FE30E94A02A9B01AC0160E070E080E022
:1017E00090E40E94032B9B01AC01C501B4010E944F
:1017F000A02A9B01AC01C701B6010E949C2A1816C1
:101800005CF5A701960160E070E08CED93EC0E941E
:10181000F52820E030E040E451E40E94F52820E083
:1018200030E040E05FE30E94A02A9B01AC0160E051
:1018300070E080E090E40E94032B9B01AC01C701A3
:10184000B6010E94A02A6093730270937402809381
:1018500075029093760213C0FE01EE0FFF1FEE0F8C
:10186000FF1FEF5AFD4F80819181A281B381809348
:10187000730290937402A0937502B0937602609104
:10188000730270917402809175029091760220919A
:101890002802309129022F3F4FEF340731F02F5F9C
:1018A0003F4F30932902209328020E947C0E6B0147
:1018B0007C0120E034E244EF51E40E94F12887FFEC
:1018C00008C086EFC82E88E2D82E84EFE82E81E487
:1018D000F82E20E030E040E051E4C701B6010E945C
:1018E000A02A9B01AC0160E074E284E79BE40E94C3
:1018F000F5286B017C010E94622970939700609328
:101900009600209106013091070140910801509105
:101910000901C701B6010E94A02A0E9462297093A2
:1019200099006093980080913C02882309F433C1A8
:10193000C0903702D0903802E0903902F0903A021D
:1019400020E030E0A901C701B6010E949C2A1816C8
:10195000D4F580912802909129028F3F2FEF9207B2
:1019600029F001969093290280932802C701B601BD
:101970000E947C0E20E030E040E051E40E94A02A6A
:101980009B01AC0160E074E284E79BE40E94F528CF
:101990006B017C010E94622970939700609396000E
:1019A00020910601309107014091080150910901F1
:1019B000C701B6010E94A02A0E9462297093990073
:1019C0006093980008C010929700109296001092B1
:1019D00099001092980060913102709132026F5F0D
:1019E0007F4F7093320260933102209196003091C4
:1019F000970080E090E0232BF1F0C0919600D09109
:101A000097000E948E296B017C01BE0180E090E06E
:101A10000E948E299B01AC016091330270913402C7
:101A200080913502909136020E94F52820E03FEF28
:101A30004FE757E410C00E948E296B017C0120E023
:101A400030EE4FEF54E46091330270913402809194
:101A50003502909136020E94A02A9B01AC01C70179
:101A6000B6010E949C2A87FD96C080912F028F5F4D
:101A700080932F0290E0209103033091040382179A
:101A80009307A0F080910E03882319F010922F0283
:101A90000DC0809171008D7F8093710080919000C6
:101AA0008F738093900010923C027DC08091300231
:101AB000C0912F02811128C0C0900803D090090363
:101AC000E0900A03F0900B0320E030E0A901C70189
:101AD000B6010E949C2A1816BCF481E08093300263
:101AE00010923702109238021092390210923A0284
:101AF000C0923302D0923402E0923502F092360264
:101B0000C150C0932F0243C010923002109229029C
:101B100010922802E0910503F091060348E0C49F6B
:101B2000E00DF11D112480819181A281B381809308
:101B3000370290933802A0933902B0933A0220E022
:101B400030E040E85EE364817581868197810E9480
:101B5000A02A6B017C0180910A01682F70E080E06F
:101B600090E00E948E2920E030E048EC52E40E9490
:101B7000F5289B01AC01C701B6010E94A02A609321
:101B800033027093340280933502909336021092A0
:101B90003202109231028091070380FD04C010923E
:101BA0003C0210923B02FF91EF91DF91CF91BF91E8
:101BB000AF919F918F917F916F915F914F913F91E5
:101BC0002F91FF90EF90DF90CF90BF90AF909F90BC
:101BD0008F907F906F905F904F900F900FBE0F90FF
:101BE0001F901895CF92DF92EF92FF92CF93DF93E1
:101BF0006B017C01EA0180912A02811102C00E94DE
:101C0000ED098091070380FF46C080917902909191
:101C10007A0208970CF03FC0809171008D7F80930D
:101C2000710080913C0281110E94070A81E080933B
:101C30003B02109229021092280220E030E0A90114
:101C4000C701B6010E949C2A1816DCF48091790223
:101C500090917A02FC01EE0FFF1FEE0FFF1FEF5A6B
:101C6000FD4FC082D182E282F382FC01EE0FFF1FA2
:101C7000EF5BFD4FD183C083019690937A028093EE
:101C80007902809171008260809371008091900050
:101C9000806880939000DF91CF91FF90EF90DF906C
:101CA000CF90089580910703817008958091070374
:101CB0008160809307030E94AA230C94D203809131
:101CC00007038E7F809307030C94AA2380917B02E5
:101CD00090E0019666E070E00E946E2C80937B029B
:101CE000089580917B0290E0019766E070E00E9489
:101CF0006E2C80937B0208958F929F92AF92BF9239
:101D0000CF92DF92EF92FF920F931F93CF93DF93C7
:101D10006B017C01C0912802D0912902BE0180E0B4
:101D200090E00E948E294B015C01A701960160E0C2
:101D300070E08CE594E40E94F5289B01AC01C5019C
:101D4000B4010E94A02A0E94622920917B022330C4
:101D500009F473C028F4222351F02130E9F02CC19A
:101D6000243009F4A0C0253009F4E0C025C180E08A
:101D700090E0A0E0BFE38093060190930701A09359
:101D80000801B093090110922B0210922C021092BC
:101D90002D0210922E0210C110922B0210922C02D2
:101DA00010922D0210922E026431710540F46A30B7
:101DB000710560F520E030E040E85EE32BC0693C4F
:101DC000710508F0AAC080E090E00E948E2920E012
:101DD00030E040EA51E40E948C2820E030E044E307
:101DE00053E40E94F5289B01AC010E94A02A20E048
:101DF00030E040E05EE30E94A02A9B01AC0160E07D
:101E000070E080E09EE30E948C2844C020E030E037
:101E100040E05FE3C701B6010E94A02A6B017C018C
:101E200080E090E0A0E0BEE380930601909307017C
:101E3000A0930801B0930901BFC010922B02109229
:101E40002C0210922D0210922E024AE0469F900121
:101E5000479F300D1124C90168EB7BE00E945A2C8A
:101E6000BC016C5D754077FF03C071956195710988
:101E7000882777FD8095982F0E9490292EE333ECD8
:101E80004EE259E30E94A02A20E030E040EC5EE3FD
:101E90000E948D28609306017093070180930801CA
:101EA0009093090189C010922B0210922C0210927B
:101EB0002D0210922E02CE0183709927892BE1F01A
:101EC000BE016170772780E090E00E948E2920E0BB
:101ED00030E040E05EE30E94A02A20E030E040E4F1
:101EE0005FE30E948D286093060170930701809341
:101EF0000801909309010CC080E090E0A0E0BFE3EE
:101F00008093060190930701A0930801B093090103
:101F1000C770DD27CD2B09F04FC01092060110923B
:101F20000701109208011092090146C010922B027D
:101F300010922C0210922D0210922E0200E010E05E
:101F400020E03FE30093060110930701209308016E
:101F5000309309016739710578F180E090E00E94C3
:101F60008E2920E030E047E153E40E948C2820E0F5
:101F700030E04AE754E40E94F52820E030E048E4ED
:101F800052E40E94A02A20E030E040EA51E40E949E
:101F9000D2290E945D29660F771F660F771FFB010C
:101FA000EE5AFE4F2081318142815381C701B60133
:101FB0000E94A02A6B017C01C701B601DF91CF917D
:101FC0001F910F91FF90EF90DF90CF90BF90AF9057
:101FD0009F908F90089580918C020895CF93DF9306
:101FE00000D01F92CDB7DEB79C01809113038430DF
:101FF00019F593E099833B832A839093E9008FEF4F
:102000009091E800815095FD06C095ED9A95F1F705
:1020100000008111F5CF8091E80085FF0DC040E000
:1020200050E063E070E0CE0101960E944F12809173
:10203000E8008E778093E8000F900F900F90DF916B
:10204000CF910895CF93DF9300D01F92CDB7DEB725
:1020500020911303243021F522E029839B838A8376
:1020600083E08093E9008FEF9091E800815095FD27
:1020700006C095ED9A95F1F700008111F5CF80919A
:10208000E80085FF0DC040E050E063E070E0CE0165
:1020900001960E944F128091E8008E778093E800AD
:1020A0000F900F900F90DF91CF910895209113031F
:1020B0002430F1F422E02093E9002FEF3091E80082
:1020C000215035FD06C035ED3A95F1F7000021119C
:1020D000F5CF2091E80025FF0BC040E050E065E01F
:1020E00070E00E944F128091E8008E778093E800A4
:1020F0000895CF93DF93EC0190911303943009F08E
:1021000046C0809115018823D9F08091160188235B
:10211000B9F09093E9008FEF9091E800815095FD20
:1021200006C095E19A95F1F700008111F5CF8091F5
:10213000E80085FF2CC040E050E060E170E017C08F
:1021400081E08093E9008FEF9091E800815095FD48
:1021500006C095ED9A95F1F700008111F5CF8091B9
:10216000E80085FF14C040E050E068E070E0CE0178
:102170000E944F128091E8008E778093E80080E102
:10218000FE01ACE7B2E001900D928A95E1F7DF9194
:10219000CF91089580911203811109C00E94E41328
:1021A0000E9441148091E20084608093E2000895CF
:1021B000109212030895089508950C94882242E025
:1021C00061EC81E00E945E1342E061EC82E00E94DB
:1021D0005E1342E061EC83E00E945E1342E161EC39
:1021E00084E00C945E1380911503833009F455C08C
:1021F00030F4813071F0823009F48EC008958A3055
:1022000009F47AC08B3009F460C0893009F09CC0B1
:1022100020C080911403813A09F096C08091E800B3
:10222000877F8093E8008091180390911903892B90
:1022300021F460E18CE792E003C060E080E090E090
:1022400070E00E949A128091E8008B778093E800FA
:10225000089580911403813209F076C080911803AB
:1022600090911903009719F0039709F06DC08091C0
:10227000E800877F8093E8008091E80082FD05C038
:10228000809113038111F8CF5FC08091F10080939A
:102290008C028091E8008B7753C080911403813ABF
:1022A00009F052C08091180390911903892B09F00D
:1022B0004BC08091E800877F8093E8008091E80020
:1022C00080FFFCCF8091150136C0809114038132CC
:1022D000D9F58091180390911903892BA9F5809164
:1022E000E800877F8093E8000E9493138091160393
:1022F000809315010C94C91B80911403813221F540
:102300008091E800877F8093E8000E94931380917A
:10231000170380938D02089580911403813AA1F4EC
:102320008091E800877F8093E8008091E80080FF3B
:10233000FCCF80918D028093F1008091E8008E7730
:102340008093E8000C949313089584B7877F84BF2B
:1023500088E10FB6F89480936000109260000FBE81
:1023600090E080E80FB6F89480936100909361004C
:102370000FBE0E9436170E94E4130E944114809100
:10238000E20084608093E20078940E94C7160E9465
:1023900038178BE091E00E94E2168091130385309C
:1023A00069F40E944922809111038823B1F30E94AD
:1023B0007722882391F30E943912EFCF0E944017B1
:1023C000ECCF292F332723303105C9F064F42130B5
:1023D000310581F02230310509F043C08DE690E0EF
:1023E00020E833E042C021323105F1F022323105DC
:1023F00041F137C082E190E02DEE33E036C09927FD
:102400008130910541F08230910541F0892B49F5E9
:10241000ECE7F3E005C0EEE4F3E002C0E4E2F3E051
:10242000849190E09F0121C06430D8F4E62FF0E061
:10243000EE0FFF1FE255FE4F2081318189E090E0D1
:1024400014C0643070F470E0FB01EE0FFF1FEA551A
:10245000FE4F20813181FB01EE55FE4F808190E0DF
:1024600004C080E090E020E030E0FA013183208376
:10247000089580E189BD82E189BD09B400FEFDCFE8
:102480008091D8008F7D8093D8008091E000826099
:102490008093E0008091E00081FDFCCF0895CF9211
:1024A000DF92EF92FF920F931F93CF93DF93EC0194
:1024B0008B016A010E94B213811133C0C114D1048F
:1024C00039F0F60180819181081B190BC80FD91FC3
:1024D000E12CF12C0115110519F18091E80085FD21
:1024E00016C08091E8008E778093E800C114D10473
:1024F00049F0F60180819181E80EF91EF182E082B7
:1025000085E00FC00E94B213882321F30AC089918D
:102510008093F10001501109FFEFEF1AFF0ADACFA3
:1025200080E0DF91CF911F910F91FF90EF90DF90AE
:10253000CF90089520911A0330911B032617370777
:1025400048F06115710539F42091E8002E77209349
:10255000E80001C0B90140E061157105A9F12091C1
:102560001303222309F443C0253009F442C020910B
:10257000E80023FD40C02091E80022FD32C02091F8
:10258000E80020FFE9CF4091F3002091F20030E015
:10259000342BFC01CF016115710559F0283031054C
:1025A00040F481918093F100615071092F5F3F4F9A
:1025B000F1CF41E02830310509F040E02091E800FA
:1025C0002E772093E800C8CF4111C9CF0AC080916F
:1025D0001303882361F0853061F08091E80083FD6A
:1025E0000AC08091E80082FFF2CF80E0089582E087
:1025F000089583E0089581E0089520911A033091B1
:102600001B032617370748F06115710539F420912F
:10261000E8002E772093E80001C0B901FC0120E01A
:102620006115710591F180911303882309F440C06D
:10263000853009F43FC08091E80083FD3DC0809162
:10264000E80082FD2FC08091E80080FFE9CF209153
:10265000F3008091F20090E0922B6115710559F022
:102660008830910540F424912093F1003196615017
:1026700071090196F2CF21E0089709F020E08091DE
:10268000E8008E778093E800CBCF2111CCCF0AC031
:1026900080911303882361F0853061F08091E80018
:1026A00083FD0AC08091E80082FFF2CF80E00895A8
:1026B00082E0089583E0089581E00895982F97308F
:1026C00058F59093E900981739F07091EC0020913B
:1026D000ED005091F00003C0242F762F50E021FF31
:1026E00019C03091EB003E7F3093EB003091ED004C
:1026F0003D7F3093ED003091EB0031603093EB0083
:102700007093EC002093ED005093F0002091EE00C8
:1027100027FF07C09F5FD3CF8F708093E90081E0D0
:10272000089580E008958091140387FF11C080917F
:10273000E80082FD05C0809113038111F8CF11C01C
:102740008091E8008B770BC080911303882349F0B8
:102750008091E80080FFF8CF8091E8008E77809329
:10276000E80008952091E4003091E50095E640915D
:10277000EC00842F817040FF22C08091E80080FD32
:102780001CC080911303882391F0853091F08091D3
:10279000EB0085FD10C04091E4005091E500421728
:1027A000530729F39A01915011F784E0089582E0CC
:1027B000089583E0089581E0089580E008954091B0
:1027C000E80042FFDECF08950E9452140E945A147E
:1027D000E0EEF0E0808181608083E8EDF0E08081D0
:1027E0008F77808319BCA7EDB0E08C918E7F8C939E
:1027F00080818F7E80831092120308950F931F9320
:10280000CF93DF930E9452140E945A14C8EDD0E077
:1028100088818F77888388818068888388818F7D8D
:10282000888319BC1092130310920F0310921103A6
:102830001092100300EE10E0F80180818B7F8083FE
:1028400088818160888342E060E080E00E945E13BE
:10285000E1EEF0E080818E7F8083E2EEF0E0808127
:1028600081608083808188608083F80180818E7F91
:102870008083888180618883DF91CF911F910F9140
:102880000895E8EDF0E080818F7E8083E7EDF0E051
:1028900080818160808384E082BF81E08093120325
:1028A0000C94FE13E8EDF0E080818E7F808310921F
:1028B000E20008951092DA001092E10008951F924C
:1028C0000F920FB60F9211242F933F934F935F9364
:1028D0006F937F938F939F93AF93BF93EF93FF93E8
:1028E0008091E10082FF0BC08091E20082FF07C06F
:1028F0008091E1008B7F8093E1000E94C616809159
:10290000DA0080FF1FC08091D80080FF1BC080913B
:10291000DA008E7F8093DA008091D90080FF0DC0AD
:1029200080E189BD82E189BD09B400FEFDCF81E06F
:10293000809313030E94CA1005C019BC10921303A0
:102940000E94D8108091E10080FF19C08091E200C0
:1029500080FF15C08091E2008E7F8093E20080911D
:10296000E20080618093E2008091D80080628093D1
:10297000D80019BC85E0809313030E94DC1080917D
:10298000E10084FF30C08091E20084FF2CC080E130
:1029900089BD82E189BD09B400FEFDCF8091D800D8
:1029A0008F7D8093D8008091E1008F7E8093E1003D
:1029B0008091E2008F7E8093E2008091E20081604E
:1029C0008093E20080910F03882311F084E007C018
:1029D0008091E30087FD02C081E001C083E0809325
:1029E00013030E94DD108091E10083FF29C08091D4
:1029F000E20083FF25C08091E100877F8093E100A2
:102A000082E08093130310920F038091E1008E7F88
:102A10008093E1008091E2008E7F8093E2008091BC
:102A2000E20080618093E20042E060E080E00E948A
:102A30005E138091F00088608093F0000E94DB10AC
:102A4000FF91EF91BF91AF919F918F917F916F9186
:102A50005F914F913F912F910F900FBE0F901F905C
:102A600018951F920F920FB60F9211242F933F9338
:102A70004F935F936F937F938F939F93AF93BF9386
:102A8000CF93DF93EF93FF93C091E900CF708091D4
:102A9000EC00D82FD17080FDD0E81092E900809131
:102AA000F000877F8093F00078940E947515109253
:102AB000E9008091F00088608093F000CD2BCF700A
:102AC000C093E900FF91EF91DF91CF91BF91AF915A
:102AD0009F918F917F916F915F914F913F912F9136
:102AE0000F900FBE0F901F9018951F93CF93DF93F9
:102AF000CDB7DEB7AA970FB6F894DEBF0FBECDBF35
:102B0000E4E1F3E088E08E0F9091F10091938E1351
:102B1000FBCF0E94F3108091E80083FF1FC18091DA
:102B2000140390911503492F50E04A30510508F0E5
:102B300015C1FA01EA5AFF4F0C94822C803881F0BB
:102B4000823809F00BC1809118038F708093E900DF
:102B50008091EB0085FB882780F91092E90006C080
:102B60008091100390911103911182609091E8007F
:102B7000977F9093E8008093F1001092F100C8C015
:102B8000282F2D7F09F0EAC0882319F0823061F0E8
:102B9000E5C080911603813009F0E0C0933009F060
:102BA00080E0809311032BC080911603811127C010
:102BB000809118038F7009F4D1C08093E9002091AF
:102BC000EB0020FF1CC0933021F48091EB00806269
:102BD00014C09091EB0090619093EB0021E030E005
:102BE000A90102C0440F551F8A95E2F74093EA00FD
:102BF0001092EA008091EB0088608093EB001092C5
:102C0000E9008091E800877F86C08111A7C01091FC
:102C100016031F778091E3008078812B8093E30077
:102C20008091E800877F8093E8000E949313809151
:102C3000E80080FFFCCF8091E30080688093E30090
:102C4000111102C082E001C083E08093130386C0AB
:102C50008058823008F082C080911603909117034B
:102C60008C3D53E0950779F583E08A838AE2898376
:102C70004FB7F894DE01139620E03EE051E2E32FD7
:102C8000F0E050935700E49120FF03C0E295EF700D
:102C90003F5FEF708E2F90E0EA3010F0C79601C0D2
:102CA000C0968D939D932F5F243149F74FBF80913C
:102CB000E800877F8093E8006AE270E0CE01019629
:102CC0000E949A1214C0AE014F5F5F4F60911803CB
:102CD0000E94E111BC01009709F440C09091E80006
:102CE000977F9093E80089819A810E94FD128091DC
:102CF000E8008B778093E80031C0803879F58091C7
:102D0000E800877F8093E80080910F038093F100B3
:102D10008091E8008E778093E8000E9493131EC094
:102D200081111CC0909116039230C0F48091E8008C
:102D3000877F8093E80090930F030E949313809104
:102D40000F03811106C08091E30087FD02C081E07E
:102D500001C084E0809313030E94DF108091E8009B
:102D600083FF0AC08091E800877F8093E80080910C
:102D7000EB0080628093EB00AA960FB6F894DEBF5A
:102D80000FBECDBFDF91CF911F9108950895CF93CE
:102D9000809113038823A1F0C091E900CF70909136
:102DA000EC00892F817090FD80E8C82B1092E9001B
:102DB0008091E80083FD0E947515CF70C093E900F3
:102DC000CF91089590939302809392020895E09199
:102DD0009202F0919302309721F00190F081E02D62
:102DE000099480E00895E0919202F0919302309767
:102DF00021F00280F381E02D09940895E091920280
:102E0000F0919302309721F00480F581E02D099430
:102E1000089520919002309191028217930771F0EA
:102E20009093910280939002E0919202F09193022C
:102E3000309721F00680F781E02D099408952091C4
:102E40008E0230918F028217930771F090938F0258
:102E500080938E02E0919202F0919302309721F0DC
:102E60000084F185E02D0994089508950C94351798
:102E70000E94BC220E940D090E9442230C94F1275B
:102E80005F926F927F928F929F92AF92BF92CF92FA
:102E9000DF92EF92FF920F931F93CF93DF9300D0B7
:102EA00000D01F92CDB7DEB70E9452099DE9C92E0E
:102EB00092E0D92E03E010E0AA24A394B12C502E66
:102EC000802F0E94CD094C01F601729062906F0133
:102ED0006826792661147104A1F40150110978F76C
:102EE0008FEF89838A831B820E94C5228160782F9D
:102EF0009D838C8349815A816B818D810E94F0175B
:102F000038C08091F20281FD0E94D6092BE030E0AA
:102F10007501022E02C0EE0CFF1C0A94E2F7C701F5
:102F200086219721892B09F129835A828E209F209F
:102F300091E0892809F490E09B830E94C52281607A
:102F4000782F9D838C8349815A816B818D810E946A
:102F5000F017000F111FF801EB56FD4F8081918192
:102F6000E826F926F182E08204C02150310980F67A
:102F7000B4CF0E942925109194020E94E7161817D9
:102F8000D1F00E94E716809394020F900F900F905B
:102F90000F900F90DF91CF911F910F91FF90EF90C5
:102FA000DF90CF90BF90AF909F908F907F906F9069
:102FB0005F900C94F7080F900F900F900F900F9068
:102FC000DF91CF911F910F91FF90EF90DF90CF9005
:102FD000BF90AF909F908F907F906F905F9008957B
:102FE000CF93DF93CDB7DEB72B970FB6F894DEBF44
:102FF0000FBECDBF4F83588769877A878B87DE01E5
:10300000119686E0FD0111928A95E9F785E0FE01AF
:10301000379601900D928A95E1F749815A816B812B
:103020007C818D819E810E94671E2B960FB6F8943D
:10303000DEBF0FBECDBFDF91CF910895CF93882320
:1030400009F4C2C0C82F823859F40E94E71681FDE6
:10305000BBC089E30E9441210E940E2289E30CC07B
:10306000833879F40E94E71680FDAEC083E50E94A4
:1030700041210E940E2283E50E948321CF910C946E
:103080000E22843859F40E94E71682FD9DC087E421
:103090000E9441210E940E2287E4EECF8CEF8C0F1C
:1030A000813A48F48C2F0E94592781118DC08C2FB2
:1030B0000E944121E3CF80E28C0F883048F4C77032
:1030C00081E001C0880FCA95EAF70E94C721D6CFD8
:1030D0008BE58C0F833078F4C53A29F0C63A31F08D
:1030E00083E890E005C081E890E002C082E890E0CB
:1030F000CF910C94091788E58C0F833108F064C0D8
:10310000C83A39F1C93A41F1CA3A49F1CB3A51F1D9
:10311000CC3A59F1CD3A61F1C03B69F1CE3A71F147
:10312000CF3A79F1C13B81F1C23B89F1C33B91F1C7
:10313000C43B99F1C53BA1F1C63BA9F1C73BB1F135
:10314000C83BB9F1C93BC1F1CA3BC9F180E090E08D
:1031500038C082EE90E035C089EE90E032C08AEE51
:1031600090E02FC085EB90E02CC086EB90E029C06A
:1031700087EB90E026C08CEC90E023C08DEC90E0D3
:1031800020C083E891E01DC08AE891E01AC082E97E
:1031900091E017C084E991E014C081E292E011C08F
:1031A00083E292E00EC084E292E00BC085E292E0FE
:1031B00008C086E292E005C087E292E002C08AE29F
:1031C00092E0CF910C941F17CF910895882309F4B2
:1031D0004BC0823859F40E94E71681FF45C089E34D
:1031E0000E9441210E940E2289E30CC0833871F4B1
:1031F0000E94E71680FF38C083E50E9441210E94AB
:103200000E2283E50E9483210C940E22843859F407
:103210000E94E71682FF28C087E40E9441210E9495
:103220000E2287E4EFCF9CEF980F913A58F390E28B
:10323000980F983050F4877091E001C0990F8A95EB
:10324000EAF7892F0E94CD21DFCF9BE5980F9330BD
:1032500020F480E090E00C940917885A833120F420
:1032600080E090E00C941F170895882321F00E94BD
:10327000C7210C940E220895882321F00E94CD21AD
:103280000C940E2208957F928F929F92AF92BF92DC
:10329000CF92DF92EF92FF920F931F93CF93DF9322
:1032A0001F92CDB7DEB77C01C62E772EFC010581BB
:1032B00002950F70128111110E94E4210E943A219F
:1032C000882379F0112369F080E28C0D883048F072
:1032D00082E00E9423210E943A2191E0D82ED92633
:1032E00001C0D12CE72DE295EF70F0E0E05AFF4FDE
:1032F0000C94822C872D807F072D0F70882311F06E
:103300000295007F112389F0002309F499C180E21E
:103310008C0D883020F4802F0E94C72103C0802F9D
:103320000E94D7210E940E228BC18C2D0E94E6188C
:10333000002309F4C3C180E28C0D883020F4802F73
:103340000E94CD2103C0802F0E94DD210E940E2209
:10335000B5C1872D807F972D9F70803211F4892F02
:1033600003C0892F8295807FCC2021F0F1E0CF1619
:10337000A1F01DC0112339F0002319F1013009F526
:103380000E94F7219BC1002319F0013009F496C176
:1033900089830E94FA21898110C1112321F006300E
:1033A00008F08CC10EC0053008F088C106C1112399
:1033B00059F0002331F0F701958190FF41C19F70D2
:1033C00095830E9435197AC1002309F4F6C03EC1E5
:1033D000872D86958695837090E0009719F0019768
:1033E00061F06CC1112321F08C2D972D937002C0D8
:1033F00080E090E00E94091761C1112321F08C2D1B
:10340000972D937002C080E090E00E941F1756C174
:103410008C2D112319F00E94312402C00E9499249E
:103420000E941E254BC1872D837009F052C01111D7
:1034300045C18C2D829586958770880F880F9C2DAD
:103440009F70892E912CA12CB12C082E04C0880CC1
:10345000991CAA1CBB1C0A94D2F7C4FE14C00FE02E
:1034600010E020E030E0B901A80104C0440F551F6E
:10347000661F771F8A95D2F7CB01BA0160957095C8
:103480008095909503C060E070E0CB01272D2695D4
:103490002695237030E02230310569F02330310564
:1034A00089F0682979298A299B292130310571F011
:1034B0000E94AF1F03C1682979298A299B290E948C
:1034C000CB1FFCC00E94AF1FC501B4010E94931F17
:1034D000F5C0112319F0872D817001C086958823CE
:1034E00009F4ECC08C2D829586958770880F880F23
:1034F0009C2D9F70892E912CA12CB12C082E04C0DC
:10350000880C991CAA1CBB1C0A94D2F7C4FE14C0D8
:103510000FE010E020E030E0B901A80104C0440F42
:10352000551F661F771F8A95D2F7CB01BA016095A8
:1035300070958095909503C060E070E0CB01272DD9
:10354000269526952370422F50E04230510569F0B0
:103550004330510589F0682979298A299B2941300E
:10356000510571F00E948920A9C0682979298A290A
:103570009B290E94A520A2C00E948920C501B401F8
:103580000E946D209BC08C2D90E0FC01E05EF10953
:10359000E531F10508F050C0E059FF4F0C94822C42
:1035A0000C2D0F70872D8F71112321F00E940620A2
:1035B000802F07CF0E942720802F0E943C197EC0B9
:1035C000112341F0053008F079C0872D8F710E94DA
:1035D0004C2074C0063008F071C0F7CF112339F0C9
:1035E000872D8F710E94062069C01123C9F3872D92
:1035F0008F710E94272062C0112329F0872D8F71BF
:103600000E94F11F5BC00E94E71F58C0112351F0B8
:10361000172D1F71812F0E94062063E0812F0E94C9
:103620001A214CC081E00E942321023008F446C0D8
:1036300082E00E94232142C0112331F0002381F255
:103640008C2D0E941E183AC0002389F28C2D0E94F6
:10365000E61834C0472D4F706C2DC7010E94D50568
:103660000E940B1F2BC0111129C0472D4F7050E035
:1036700042305105B9F04CF44115510581F041300B
:103680005105E1F40E94192819C04330510569F031
:103690004430510599F48C2D0E946B280FC00E9474
:1036A00002280CC00E94352809C00E94482806C084
:1036B000472D4F706C2DC7010E94D805DD20F9F011
:1036C0000E94162180FD1BC0F70112820E9410216A
:1036D0000E940620C7010E948E1B0E9410210F909D
:1036E000DF91CF911F910F91FF90EF90DF90CF90DE
:1036F000BF90AF909F908F907F900C9427200F9059
:10370000DF91CF911F910F91FF90EF90DF90CF90BD
:10371000BF90AF909F908F907F9008950F931F93CD
:10372000CF93DF93EC01888199812B813C81232BFE
:10373000B9F09F3F11F48F3F99F0CE010E94D4035E
:10374000882371F0688179818A810E940C218C0123
:103750000E94C1200E94881FB801CE010E94431917
:10376000DF91CF911F910F9108950E94E4210E9453
:10377000F4210E94B9210E940E220E94CF250E94AE
:103780001E2580E090E00E94091780E090E00C94F4
:103790001F170E94D4210C94B51B0E940121292FD0
:1037A00022952F7030E02C3031054CF42A30310551
:1037B0006CF42250310922303105A8F407C02C30B6
:1037C000310569F02F30310551F00DC0803F69F0AF
:1037D00018F4803E40F409C0843F29F406C093FBEE
:1037E000882780F9089580E0089581E00895CF93B7
:1037F000DF9300D000D01F92CDB7DEB70F900F90AF
:103800000F900F900F90DF91CF910895CF93DF939A
:1038100000D000D000D0CDB7DEB726960FB6F89412
:10382000DEBF0FBECDBFDF91CF9108951F93CF9321
:10383000DF93C0919D0216E080919E02C81799F017
:10384000D0E01C9FF0011D9FF00D1124E156FD4FAB
:103850004081518162817381848195810E94061C1F
:103860002196C770E9CFDF91CF911F9108954091C4
:10387000CF025091D0026091D1027091D20280911A
:10388000D3029091D4020C94061C8091D4028295AC
:103890008F7009F054C08091D102882309F44FC081
:1038A00080919D02A0919E026091CF027091D00202
:1038B0004091D2025091D302B6E08A1709F43FC07A
:1038C00090E041155105C1F17F3F11F46F3FA1F127
:1038D000B89FF001B99FF00D1124E156FD4F2181F1
:1038E00072132AC02081621327C02281211124C0B3
:1038F000238134812417350710F421503109241B0A
:10390000350B283C3105C0F42091D4022F70206182
:103910002093D40226E0289FF001299FF00D112466
:10392000EC55FD4F80818F70806180838FEC92E039
:103930000E948E1B0C94161C01968770BECF0895B2
:10394000CF92DF92EF92FF920F931F93CF93DF936B
:10395000CDB7DEB762970FB6F894DEBF0FBECDBF0E
:103960008C0185E0F801DE011D9601900D928A958B
:10397000E1F7D8014C9111965C91119712966C91D8
:1039800012971396CD90DC9014973091CF027091DE
:10399000D0028091D2029091D302009709F46BC1BA
:1039A0007F3F19F43F3F09F466C1E090D102EE2059
:1039B00009F4C0C02091D402C816D90628F0F60137
:1039C000E81BF90BCF0104C0809590958C0D9D1DCF
:1039D000FF24F394883C910578F0F12C207F09F0C6
:1039E000C6C07C2DD98AC88A89890E94F71B8FECB2
:1039F00092E00E948E1BB1C0822F807F09F046C0EA
:103A0000751314C0341312C0611110C02F702061DF
:103A10002093D4020E94371C8FEC92E00E948E1BF0
:103A20008091D402D80115968C932EC0CD2819F11F
:103A30005F3F11F44F3FF9F0F62E61111CC08091E9
:103A40009D0220919E0236E0821709F45AC090E050
:103A5000389FF001399FF00D1124E156FD4F71811F
:103A6000571306C07081471303C07281711103C0E0
:103A700001968770E9CFF62E662309F418C180916C
:103A8000D40281608093D402F12C11C1751308C057
:103A9000341306C0611104C08091D402D801C3C0A0
:103AA0004D875E878D859E856A8B0E94CD1B6A89B6
:103AB0008823E1F16623D1F12091D402822F8295EF
:103AC0008F7090E0029774F08091CF029091D002B5
:103AD00098878F831986DB86CA862C87CE01079646
:103AE0000E948E1B86E0F801AFECB2E001900D92CF
:103AF0008A95E1F70E94451C0E94371CFF24F3942D
:103B0000D6C04D875E878D859E850E940121292F15
:103B100022952F7030E0223031050CF0BCC09F7030
:103B200009F0B6C0805E883008F4C1C0C8010E94A8
:103B30008E1BE4CFC816D90608F453C0F601E81B63
:103B4000F90BCF01883C910508F450C0F12C7C2D75
:103B5000D98AC88A89890E94F71BEFECF2E086E0D7
:103B6000DF011D928A95E9F70E94371CA0C07513EA
:103B700014C0341312C0611110C08091D402F80136
:103B80008583C8010E948E1B86E0EFECF2E0DF0126
:103B90001D928A95E9F7FE2C8AC04D875E878D8538
:103BA0009E856A8B0E94CD1B6A89882309F4BECF4B
:103BB000662309F4BBCF2091D402822F82958F70A7
:103BC00090E002970CF48ECF8091CF029091D002BA
:103BD0009A8389831B82DD82CC822E83CE0101965B
:103BE0007FCF809590958C0D9D1DACCFF62E6623D2
:103BF00009F49CCF75132EC034132CC02091D4022D
:103C000020FD1FC0822F82958F70D9F0D8011596A4
:103C10002C9315978F3049F08F5F982F9295907F56
:103C2000822F8F70892B15968C93C8010E948E1B52
:103C300086E0F801AFECB2E001900D928A95E1F7D1
:103C400093CF86E0F801AFECB2E001900D928A9537
:103C5000E1F72DC04D875E878D859E850E94CD1B27
:103C6000811140CF8091D40281608093D402C80139
:103C70000E948E1B1CC0662309F458CF4D875E87B7
:103C80008D859E850E94CD1B882309F44FCF2ACFB6
:103C9000811148CF0CC0243031050CF047CF9F7004
:103CA00009F440CFF8019581907F09F03BCF8F2D2B
:103CB00062960FB6F894DEBF0FBECDBFDF91CF91F5
:103CC0001F910F91FF90EF90DF90CF9008951F9379
:103CD000CF93DF93CDB7DEB72C970FB6F894DEBF46
:103CE0000FBECDBF4F83588769877A878B879C87A4
:103CF000CE0107960E94A01C882369F08F819885C9
:103D00002A853B85232BF1F19F3F09F063C08F3F4C
:103D100009F060C037C086E0FE013796DE011196DB
:103D200001900D928A95E1F76F817885EA85FB8590
:103D3000309741F17F3F11F46F3F21F120919E02B6
:103D400030E0C90101968770992740919D0250E0AB
:103D50008417950709F447C069837A83FD83EC8350
:103D600096E0929FD001939FB00D1124A156BD4FB4
:103D7000FE01319601900D929A95E1F780939E0293
:103D80000E94161C16E080919D0290919E02891758
:103D9000C1F1189FC001112481569D4F0E94A01CA3
:103DA000882379F1E0919D021E9FF0011124E156D4
:103DB000FD4F4081518162817381848195810E9490
:103DC000061C80919D0290E0019687709927809350
:103DD0009D02D9CF4F81588569857A858B859C85D1
:103DE0000E94061CCFCF0E94C91B10929E02109207
:103DF0009D02EFECF2E086E0DF011D928A95E9F783
:103E0000C1CF2C960FB6F894DEBF0FBECDBFDF91A9
:103E1000CF911F910895EF92FF920F931F93CF932D
:103E2000DF938C01009709F46CC0F12CEE24E3942D
:103E3000E8012196F8018491843740F4843008F039
:103E400051C0813081F0823019F15BC0853709F4AF
:103E500044C0A8F19CE7980F903708F052C08F77C4
:103E60000E94E61841C00E5F1F4FFE01C49180E220
:103E70008C0F883048F4C7708E2D01C0880FCA950A
:103E8000EAF70E94E72114C08C2F0E941E182DC053
:103E90000E5F1F4FFE01C49180E28C0F883058F4F2
:103EA000C7708E2D01C0880FCA95EAF70E94ED21D8
:103EB0000E940E221AC08C2F0E94E61816C00E5FB8
:103EC0001F4FFE01C491CC2381F08FE99FE0019741
:103ED000F1F700C00000C150F6CF0E5F1F4FFE018A
:103EE000F49003C00E941E188E018F2D882309F4C0
:103EF0009FCFEFE9FFE03197F1F700C0000081505C
:103F0000F5CFDF91CF911F910F91FF90EF90089522
:103F100008956093D9027093DA028093DB02909344
:103F2000DC020C94B51B0F931F930091D9021091E2
:103F3000DA022091DB023091DC02DC01CB01802B24
:103F4000912BA22BB32B8093D9029093DA02A093EA
:103F5000DB02B093DC021F910F910C94B51B0F9301
:103F60001F930091D9021091DA022091DB02309167
:103F7000DC02DC01CB0180239123A223B3238093B5
:103F8000D9029093DA02A093DB02B093DC021F9176
:103F90000F910C94B51B0F931F930091D9021091B0
:103FA000DA022091DB023091DC02DC01CB018027B8
:103FB0009127A227B3278093D9029093DA02A09386
:103FC000DB02B093DC021F910F910C94B51B109291
:103FD000D5021092D6021092D7021092D8020C94F9
:103FE000B51B41E050E060E070E004C0440F551F95
:103FF000661F771F8A95D2F74093D5025093D60259
:104000006093D7027093D8020C94B51B41E050E046
:1040100060E070E004C0440F551F661F771F8A954B
:10402000D2F78091D5029091D602A091D702B0919B
:10403000D802482B592B6A2B7B2B4093D5025093E7
:10404000D6026093D7027093D8020C94B51B41E05E
:1040500050E060E070E004C0440F551F661F771FFA
:104060008A95D2F740955095609570958091D502CC
:104070009091D602A091D702B091D802482359233B
:104080006A237B234093D5025093D6026093D702D4
:104090007093D8020C94B51B41E050E060E070E0F2
:1040A00004C0440F551F661F771F8A95D2F7809171
:1040B000D5029091D602A091D702B091D80248279C
:1040C00059276A277B274093D5025093D6026093E5
:1040D000D7027093D8020C94B51B0F931F930091D5
:1040E000D5021091D6022091D7023091D802DC017E
:1040F000CB01802B912BA22BB32B8093D5029093D5
:10410000D602A093D702B093D8021F910F910C94BE
:10411000B51B0F931F930091D5021091D6022091E9
:10412000D7023091D802DC01CB0180239123A22356
:10413000B3238093D5029093D602A093D702B09375
:10414000D8021F910F910C94B51B0F931F930091F0
:10415000D5021091D6022091D7023091D802DC010D
:10416000CB0180279127A227B3278093D502909374
:10417000D602A093D702B093D8021F910F910C944E
:10418000B51B0895CF92DF92EF92FF920F931F938A
:10419000CF93DF938C01C090D902D090DA02E090E7
:1041A000DB02F090DC028091D5029091D602A091C2
:1041B000D702B091D802C82AD92AEA2AFB2ACFE12D
:1041C000D0E0D701C6010C2E04C0B695A7959795EF
:1041D00087950A94D2F780FF06C0B8018C2F0E9401
:1041E0005D08019721F4219760F780E001C08C2FD2
:1041F000DF91CF911F910F91FF90EF90DF90CF90C3
:104200000895CF93DF93EC010E94C220BE010E946B
:104210005D08DF91CF910895CB010E94012108959F
:104220008091DD0285958595859508958091DD02C3
:104230008770089598E0899F90011124262B209380
:10424000DD020C9406202091DD028095822380936C
:10425000DD02982F977069F430E0482F552747FD0D
:1042600050952417350729F08595859585950C94EB
:10427000272008959091DD02977081E009F480E095
:10428000089590911501992321F0909116019111B3
:1042900009C02091170130911801F90132969FEF62
:1042A00040E01FC0982F9695969596959F3050F5B3
:1042B000E0911701F0911801E90FF11D877021E0DD
:1042C00030E0A90102C0440F551F8A95E2F7CA01E8
:1042D0009181892B818308959F3F39F04F5F4E3044
:1042E00041F051915813F8CF0DC05111F7CF942FD1
:1042F000F5CF9F3F39F0F901E90FF11D97FDFA95D0
:1043000082830895089590911501992321F0909149
:104310001601911109C02091170130911801F9017E
:104320003296205F3F4F1FC0982F96959695969591
:104330009F30F0F4E0911701F0911801E90FF11DA1
:10434000877021E030E0A90102C0440F551F8A9513
:10435000E2F7CA018095918189238183089531967E
:10436000E217F30729F090819813F9CF1082F7CF65
:10437000089581E090E0E0911701F0911801E80FB5
:10438000F91F1082019680319105A9F70895909147
:10439000F102892B8093F102089580959091F102AA
:1043A00089238093F10208951092F102089590916B
:1043B000F002892B8093F002089580959091F0028D
:1043C00089238093F00208951092F002089590914D
:1043D000EF02892B8093EF02089580959091EF0270
:1043E00089238093EF0208951092EF02089580933D
:1043F000DE0208951092DE020895809117019091D7
:104400001801FC0131969C01205F3F4F80E09191A3
:1044100091118F5FE217F307D1F70895E09117012B
:10442000F09118018091F1028083E0911701F091E1
:10443000180190818091F002892B8083E09117010F
:10444000F091180190818091EF02892B80838091F7
:10445000DE02882361F0E0911701F091180190814C
:10446000892B80830E94FD2181111092DE028091B0
:104470001701909118010C94F31620E0009739F081
:10448000AC0141505109842395232F5FF7CF822F30
:10449000089580911303843039F11092F30220E4DF
:1044A00088E190E00FB6F894A895809360000FBE65
:1044B0002093600080E00E94D80280E00E94F7080C
:1044C00083B7817F846083BF83B7816083BF789423
:1044D000889583B78E7F83BF88E10FB6F894809369
:1044E0006000109260000FBE08950895089580E066
:1044F0000E94D8020E9475220E9452090E947622D0
:104500000E94D70991E0811101C090E0892F0895A0
:104510000E94C91B80E00E94D8020E94F1270E94DD
:10452000E7160C94F7081F920F920FB60F92112402
:104530008F939F93AF93BF938091F302811113C028
:104540008091F4029091F502A091F602B091F702E9
:104550004196A11DB11D8093F4029093F502A093A2
:10456000F602B093F702BF91AF919F918F910F9098
:104570000FBE0F901F90189582E084BD93E095BD0B
:104580009AEF97BD80936E0008952FB7F8948091AD
:10459000F4029091F502A091F602B091F7022FBFBC
:1045A0000895CF92DF92EF92FF920F931F932FB750
:1045B000F8944091F4025091F5026091F6027091E6
:1045C000F7022FBF6A017B01EE24FF248C0120E05B
:1045D00030E0C016D106E206F30610F4415051094E
:1045E0009A01281B390BC9011F910F91FF90EF9081
:1045F000DF90CF9008951F920F920FB60F92112463
:104600008F939F93AF93BF938091F4029091F502A3
:10461000A091F602B091F7020196A11DB11D809301
:10462000F4029093F502A093F602B093F702BF91C3
:10463000AF919F918F910F900FBE0F901F90189583
:104640000E94E413F8942FEF87EA91E6215080400E
:104650009040E1F700C0000087E090EBDC01809320
:104660001E0390931F03A0932003B09321039CE0AB
:1046700088E10FB6F894A895809360000FBE9093E0
:104680006000FFCF0E948123811102C00E945D2340
:104690000E948C238093F2020E94942380931C0337
:1046A00087FB882780F9809316010E949023682F4A
:1046B00070E080E090E00C94891F6DEE7EEF80E06A
:1046C00090E00E94A82C60E082E090E00E94962C8E
:1046D00060E083E090E00E94962C60E084E090E04F
:1046E0000E94962C60E085E090E00E94962C60E0AD
:1046F00086E090E00E94962C6FEF87E090E00C94AB
:10470000962C80E090E00E94902C21E08D3E9E4F00
:1047100009F020E0822F089582E090E00C94882C2C
:1047200083E090E00C94882C84E090E00C94882C3A
:10473000682F84E090E00C94962C86E090E00C9436
:10474000882C682F86E090E00C94962C87E090E00F
:104750000C94882C682F87E090E00C94962C809124
:10476000FA0280FF0BC060911C0185E0689FB001D8
:10477000112475956795759567952BC081FF09C0C4
:1047800060911C0185E0689FB001112475956795C3
:1047900020C082FF07C060911C0185E0689FB001C6
:1047A000112417C09091FB029923D1F060911B0155
:1047B000961788F720911C0185E0289F900111240D
:1047C000929FA001939F500D112470E0CA010E9496
:1047D0006E2C6038710540F46115710539F002C026
:1047E00065E070E0862F08958FE7089581E00895D1
:1047F0008091FA0280FF08C060911A0170E07595FF
:1048000067957595679521C081FF06C060911A0173
:1048100070E07595679519C082FF04C060911A0118
:1048200070E010C09091FB029923C1F060911901D2
:104830009617A0F780911A01899FC001112470E09A
:104840000E946E2C6038710528F46115710521F005
:10485000862F08958FE7089581E0089561E070E064
:10486000F4CF803F21F40E94AF23819504C0813FA3
:1048700029F40E94AF238093FE020895823F21F421
:104880000E94AF23819504C0833F29F40E94AF2387
:104890008093FD020895893F19F40E94F82305C012
:1048A0008A3F31F40E94F82381958093FF02089596
:1048B0008B3F21F40E94F823819504C08C3F29F49A
:1048C0000E94F823809300030895843F21F480918F
:1048D000FC02816017C0853F21F48091FC02826058
:1048E00011C0863F21F48091FC0284600BC0873F99
:1048F00021F48091FC02886005C0883F31F48091EA
:10490000FC0280618093FC0208958D3F21F4809128
:10491000FA0281600BC08E3F21F48091FA0282601E
:1049200005C08F3F29F48091FA0284608093FA02D7
:104930000895803F39F48091FE0287FF6CC0109289
:10494000FE0269C0813F29F48091FE021816BCF373
:1049500062C09091FD02823F29F497FF5CC01092E3
:10496000FD0259C0833F19F41916CCF354C0893F96
:1049700041F48091FF0218160CF04DC01092FF0216
:104980004AC08A3F29F48091FF0287FF44C0F6CFD6
:104990008B3F39F48091000387FF3DC010920003E4
:1049A0003AC08C3F29F4809100031816BCF333C041
:1049B000843F21F48091FC028E7F17C0853F21F453
:1049C0008091FC028D7F11C0863F21F48091FC0212
:1049D0008B7F0BC0873F21F48091FC02877F05C04D
:1049E000883F31F48091FC028F7E8093FC0213C0DB
:1049F0008D3F21F48091FA028E7F0BC08E3F21F40F
:104A00008091FA028D7F05C08F3F29F48091FA02D0
:104A10008B7F8093FA028091FD0281110EC08091FC
:104A2000FE0281110AC08091FF02811106C08091AF
:104A30000003811102C01092FB0208958CEF92E0F6
:104A40000E94FE160E94C5229093F9028093F802FC
:104A500008951F93CF93DF938091F8029091F9020C
:104A60000E94D122AC019091FB02992321F0209168
:104A70001D0130E006C020911E018AE0289F9001B0
:104A800011244217530708F486C08091FD02C0919B
:104A9000FE02D091FF0210910003811107C0C111E5
:104AA00076C0D11174C0111172C075C09F3F19F04A
:104AB0009F5F9093FB02181624F40E94AF2380930B
:104AC000FD028091FD0287FF05C00E94AF23819502
:104AD0008093FD021C1624F40E94AF238093FE02F3
:104AE0008091FE0287FF05C00E94AF2381958093CD
:104AF000FE026091FD02662339F1C091FE02CC23D3
:104B000019F1772767FD7095872F972F0E949029BD
:104B100023E333E343E35FE30E94A02A0E945D297D
:104B20006093FD026C2F772767FD7095872F972F75
:104B30000E94902923E333E343E35FE30E94A02A2A
:104B40000E945D296093FE021D1624F40E94F82342
:104B50008093FF028091FF0287FF05C00E94F82327
:104B600081958093FF02111624F40E94F82380930C
:104B700000038091000387FF05C00E94F823819500
:104B800080930003DF91CF911F910C941E259F3FCE
:104B900009F08ECF96CFDF91CF911F910895ECEF62
:104BA000F2E085E0DF011D928A95E9F71092FB02A1
:104BB0001092FA020895833081F128F4813059F07F
:104BC0008230D1F00895853009F449C0B8F18630BB
:104BD00009F456C0089580911E01262F30E0280F59
:104BE000311D2F3F310524F4680F60931E01089595
:104BF0008FEF80931E01089580911D01262F30E0D4
:104C0000280F311D2F3F310524F4680F60931D01DB
:104C100008958FEF80931D01089580911C01262F28
:104C200030E0280F311D2F3F310524F4680F6093C9
:104C30001C0108958FEF80931C01089580911B0142
:104C4000262F30E0280F311D2F3F310524F4680F47
:104C500060931B0108958FEF80931B01089580914D
:104C60001A01262F30E0280F311D2F3F310524F483
:104C7000680F60931A0108958FEF80931A010895C9
:104C800080911901262F30E0280F311D2F3F31056B
:104C900024F4680F6093190108958FEF8093190130
:104CA0000895833011F128F4813049F0823091F079
:104CB0000895853081F120F18630C1F10895809109
:104CC0001E01681720F4861B80931E010895109220
:104CD0001E01089580911D01681720F4861B8093A2
:104CE0001D01089510921D01089580911C016817FF
:104CF00020F4861B80931C01089510921C010895D6
:104D000080911B01681720F4861B80931B01089576
:104D100010921B01089580911A01681720F4861BD8
:104D200080931A01089510921A0108958091190133
:104D3000681720F4861B80931901089510921901B9
:104D400008950F931F93873208F048C08E3108F002
:104D50008DC0803109F477C008F5873009F461C04F
:104D600068F4863009F09DC08091F202817F8E7FC9
:104D70008093F20281E08093020394C08B3009F4A7
:104D800089C08E3009F08DC08091F20282FB22270B
:104D900020F991E0922790FB82F95EC0863109F4F8
:104DA00079C060F4813109F07CC00E94C91B9091E8
:104DB000160181E08927809316016CC0893109F4BE
:104DC00069C08B3109F06DC08091F20281FB22270E
:104DD00020F991E0922790FB81F93EC0883309F4D5
:104DE00059C050F4893209F457C0853309F454C0CE
:104DF000873209F451C055C0833409F44DC028F4FA
:104E00008A3308F44EC0895332C0883409F049C04F
:104E10000E94C91B0E94070A0E94CB030E94202304
:104E200039C09091F202892F8095817080FB90F9B2
:104E300029F0966098609093F20234C0997F977F32
:104E40009093F20227C08091F20283FB222720F97F
:104E500091E0922790FB83F98093F2029923D1F09D
:104E60008091F20281608093F20214C08D5141E082
:104E700050E060E070E08A019B0104C0000F111F48
:104E8000221F331F8A95D2F7C901B8010E94891FDA
:104E90000E94C91B81E006C061E070E080E090E004
:104EA000F5CF80E01F910F91089580E0089580E094
:104EB0000895CF93C82F80910203813069F018F0D4
:104EC0008230C9F184C0E0911701F091180180810E
:104ED000823209F07EC007C0E0911701F0911801FD
:104EE0008081823261F48C2F0E945527811104C089
:104EF0008C2F0E94A1261DC081E090E01AC08C2F4B
:104F00000E945727811114C0C43179F048F4CB3086
:104F100079F0C03109F061C082E08093020308C0DB
:104F2000C93219F0C83321F058C01092020355C09D
:104F300081E0817054C0C93291F120F5C43179F11A
:104F4000B0F4C73009F047C08EE180931E0182E3C0
:104F500080931D018AE080931C0184E180931B01F2
:104F600088E080931A0188E28093190134C0CE5101
:104F7000C63088F5EC2FF0E0EA54FE4F8081809334
:104F8000010329C0CE34E9F020F4CB3421F56AE0E6
:104F900013C0C13579F0C235F1F461E00DC08091E4
:104FA0000103882319F01092010315C081E080935A
:104FB000020315C061E006C0809101030E94DB2559
:104FC0000AC06AE0809101030E94512604C0109239
:104FD000020380E004C081E002C080E0AACFCF914C
:104FE00008950E948123811102C00E945D230E94C6
:104FF0009D2380931D0380FF02C0869501C080E041
:105000000C94D80280911D03982F9695292F30E09B
:10501000233031054CF49F5F990F8170892B81609B
:1050200080931D030E94A12380911D0386950C94FB
:10503000D80280911D03982F969591F09158990F61
:105040008170892B80931D038E7F91E009F490E09D
:1050500080911D0390FB80F980931D030E94A12382
:1050600080911D0386950C94D80280911D03982F82
:10507000909590FB80F980931D030E94A12380915D
:105080001D0380FF02C0869501C080E00C94D80209
:1050900090911D03892F86958F5F8F779170843053
:1050A00028F4880F892B80931D0302C090931D0361
:1050B00080911D038E7F91E009F490E080911D03A3
:1050C00090FB80F980931D030E94A12380911D0312
:1050D00086950C94D80220911D03922F96958927CE
:1050E000982F990F822F8170892B80931D038E7FBB
:1050F00091E009F490E080911D0390FB80F980938A
:105100001D030E94A12380911D0386950C94D80253
:1051100080911D03869508955058BB27AA270ED06D
:10512000D1C1C2D130F0C7D120F031F49F3F11F48A
:105130001EF4B7C10EF4E095E7FB9FC1E92FD3D170
:1051400080F3BA17620773078407950718F071F4A4
:105150009EF5EBC10EF4E0950B2EBA2FA02D0B019E
:10516000B90190010C01CA01A0011124FF27591BAC
:1051700099F0593F50F4503E68F11A16F040A22FB2
:10518000232F342F4427585FF3CF46953795279523
:10519000A795F0405395C9F77EF41F16BA0B620B22
:1051A000730B840BBAF09150A1F0FF0FBB1F661F69
:1051B000771F881FC2F70EC0BA0F621F731F841FAC
:1051C00048F4879577956795B795F7959E3F08F0D2
:1051D000B3CF9395880F08F09927EE0F9795879591
:1051E000089527D108F481E008950CD06BC163D1F4
:1051F00040F05AD130F021F45F3F19F03EC1511117
:1052000095C14FC170D198F39923C9F35523B1F3D8
:10521000951B550BBB27AA2762177307840738F025
:105220009F5F5F4F220F331F441FAA1FA9F333D084
:105230000E2E3AF0E0E830D091505040E695001C38
:10524000CAF729D0FE2F27D0660F771F881FBB1FF4
:10525000261737074807AB07B0E809F0BB0B802DCE
:10526000BF01FF2793585F4F2AF09E3F510568F01A
:1052700004C15CC15F3FECF3983EDCF38695779503
:105280006795B795F7959F5FC9F7880F911D96951C
:10529000879597F90895E1E0660F771F881FBB1F78
:1052A000621773078407BA0720F0621B730B840B25
:1052B000BA0BEE1F88F7E095089504D06894B111F9
:1052C00035C1089518D188F09F5790F0B92F9927CC
:1052D000B751A0F0D1F0660F771F881F991F1AF001
:1052E000BA95C9F712C0B13081F01FD1B1E008956D
:1052F0001CC1672F782F8827B85F39F0B93FCCF3EE
:10530000869577956795B395D9F73EF490958095F6
:10531000709561957F4F8F4F9F4F0895E89409C016
:1053200097FB3EF490958095709561957F4F8F4FD8
:105330009F4F9923A9F0F92F96E9BB279395F695EE
:10534000879577956795B795F111F8CFFAF4BB0F6C
:1053500011F460FF1BC06F5F7F4F8F4F9F4F16C0D0
:10536000882311F096E911C0772321F09EE8872F5A
:10537000762F05C0662371F096E8862F70E060E016
:105380002AF09A95660F771F881FDAF7880F96958F
:10539000879597F9089588D018F011F08CD038F4DB
:1053A00080C0C4C0E92F9FD0B0F35523C9F3E7FBF9
:1053B0006217730784079507A8F199F3E92FFF2770
:1053C00088232AF03197660F771F881FDAF7952F09
:1053D0005527442332F091505040220F331F441F71
:1053E000D2F7BB27E91BF50B621B730B840BB109CA
:1053F000C1F222F4620F731F841FB11D31972AF08E
:10540000660F771F881FBB1FEFCF915050405AF097
:1054100041F0882332F0660F771F881F915050406B
:10542000C1F7939530C08695779567959F5FD9F7BB
:10543000F8CF990F0008550FAA0BE0E8FEEF1616FB
:105440001706E807F907C0F012161306E407F50778
:1054500098F0621B730B840B950B39F40A2661F0EC
:10546000232B242B252B21F408950A2609F4A1408F
:10547000A6958FEF811D811D089597F99F6780E89C
:1054800070E060E008959F3F31F0915020F48795DF
:1054900077956795B795880F911D9695879597F99C
:1054A00008959FEF80EC089500240A9416161706BD
:1054B00018060906089500240A9412161306140605
:1054C00005060895092E0394000C11F4882352F068
:1054D000BB0F40F4BF2B11F460FF04C06F5F7F4F20
:1054E0008F4F9F4F089557FD9058440F551F59F007
:1054F0005F3F71F04795880F97FB991F61F09F3FC1
:1055000079F087950895121613061406551FF2CFE9
:105510004695F1DF08C0161617061806991FF1CF39
:1055200086957105610508940895E894BB27662760
:105530007727CB0197F908957CDF08F48FEF089562
:105540000BD0C0CFB1DF28F0B6DF18F0952309F0FB
:1055500094CFA7CF1124EACFC6DFA0F3959FD1F354
:10556000950F50E0551F629FF001729FBB27F00D11
:10557000B11D639FAA27F00DB11DAA1F649F662766
:10558000B00DA11D661F829F2227B00DA11D621FB5
:10559000739FB00DA11D621F839FA00D611D221F6F
:1055A000749F3327A00D611D231F849F600D211D53
:1055B000822F762F6A2F11249F5750408AF0E1F0F6
:1055C00088234AF0EE0FFF1FBB1F661F771F881F3F
:1055D00091505040A9F79E3F510570F04ECFA6CF95
:1055E0005F3FECF3983EDCF3869577956795B7952A
:1055F000F795E7959F5FC1F7FE2B880F911D969554
:10560000879597F90895FA01EE0FFF1F309621054F
:10561000310599F16115710561F48038BFE39B078D
:1056200049F168949038810561F08038BFEF9B079D
:1056300041F0992342F5FF3FE1053105210511F1C4
:10564000E8940894E795D901AA2329F4AB2FBE2F3B
:10565000F85FD0F310C0FF5F70F4A695E0F7F7395C
:1056600050F019F0FF3A38F49F779F930CD00F90C9
:1056700007FC905808953EF014CF60E070E080E899
:105680009FE308954FE79F775F934F933F932F9347
:105690009ED02F913F914F915F9152DF05C019F439
:1056A0000EF0EBCE42CFFDCE26DFC8F39638C0F722
:1056B00007F80F92E8942BE33AEA48EB5FE74EDFF6
:1056C0000F920F920F924DB75EB70F92C0D0EAE0E3
:1056D000F1E016D04F915F91EF91FF91E595EE1FAC
:1056E000FF1F49F0FE57E0684427EE0F441FFA956C
:1056F000E1F74195550B32D00F9007FE26C0089573
:10570000DF93CF931F930F93FF92EF92DF927B0172
:105710008C01689405C0DA2EEF011EDFFE01E894CB
:10572000A5912591359145915591AEF3EF0106DD97
:10573000FE019701A801DA9479F7DF90EF90FF90CE
:105740000F911F91CF91DF9108959B01AC0160E013
:1057500070E080E89FE349CD90CE95CECCDEE8F3B3
:105760009923D9F3940F511DBBF39150504094F0FD
:1057700059F0882332F0660F771F881F91505040F0
:10578000C1F79E3F510544F7880F911D9695879567
:1057900097F908955F3FACF0983E9CF0BB27869543
:1057A00077956795B79508F4B1609395C1F7BB0FEE
:1057B00058F711F460FFE8CF6F5F7F4F8F4F9F4F17
:1057C000E3CFB4CE0EF05FCE6CCE689456CE93DEAF
:1057D000C8F39923D1F3C6F3DF93CF931F930F93AD
:1057E000FF92C92FDD2788232AF02197660F771FA4
:1057F000881FDAF720E030E040E85FEB9FE388396C
:1058000020F0803E30F021968F7787DCE2E3F1E0F4
:1058100003C083DCEFE5F1E073DF8B01BE01EC0137
:10582000FB2E6F5771097595771F880B990B78DDE3
:1058300028E132E741E35FE38FDEAF2D9801AE014F
:10584000FF900F911F91CF91DF9178DC3BCEFA0151
:10585000DC01AA0FBB1F9B01AC01BF5728F4222714
:105860003327442750781FC0B75188F4AB2F00244A
:10587000469537952795011CA395D2F3002069F032
:10588000220F331F441FB395DAF30DD045CC61309E
:105890007105A0E88A07B94630F49B01AC01662780
:1058A000772788279078309621F0208331834283B0
:1058B00053830895AA1BBB1B51E107C0AA1FBB1F3E
:1058C000A617B70710F0A61BB70B881F991F5A958C
:1058D000A9F780959095BC01CD01089597FB072EFF
:1058E00016F4009407D077FD09D00E945A2C07FCCB
:1058F00005D03EF4909581959F4F089570956195E0
:105900007F4F0895EE0FFF1F0590F491E02D09944D
:10591000F999FECF92BD81BDF89A992780B5089577
:10592000A8E1B0E042E050E00C94B02C262FF999A9
:10593000FECF92BD81BDF89A019700B4021639F0EE
:105940001FBA20BD0FB6F894FA9AF99A0FBE0895BF
:105950000196272F0E94972C0C94962CDC01CB01EA
:10596000FC01F999FECF06C0F2BDE1BDF89A31966F
:1059700000B40D9241505040B8F70895F894FFCF0D
:10598000640007000CFF0000003F64EB0F79105625
:10599000102210EE0F0101DF022808140A321E0047
:1059A00002040507090B0C0E1011131517181A1C09
:1059B0001D1F2123242628292B2D2F303234353743
:1059C000393B1F0F03764F5F6F7F49694379095950
:1059D00053633149803F5D8B803FF8BF803FCAE110
:1059E000803F73ED803FCAE1803FF8BF803F5D8B11
:1059F000803F3149803F0000803FF16D7F3F75EA75
:105A00007E3F4C827E3F833F7E3F84287E3F833FA4
:105A10007E3F4C827E3F75EA7E3FF16D7F3F000006
:105A2000803F3F4D3639BB046E043804FF039203B8
:105A3000AB03C403DD0301020304050607080900E4
:00000001FF
